:020000040000FA
:020000007D2859
:080008000000F800030E830163
:10001000F9000A08FA008A010408FB00831203139E
:10002000101083120313BF308E00EE308F00831246
:100030000313FC03031D1F28FD0AC830FC00043015
:10004000A006201D2C2823080F398A110A12002728
:100050008038870086133328230E0F398A110A123D
:10006000002787008617831203130C1083160313CF
:100070000C14831203131014831203137B088400DF
:100080007A088A00790E8300F80E780E0900831230
:1000900003130B178B178312031300308312031300
:1000A000C830FC00831203130C10831603130C14C6
:1000B00083120313101483120313FD01A101A20183
:1000C0000030A5000130A40008008312031385014D
:1000D0008601FF308700831203179E0183120317E6
:1000E0009F01831603130B3085007F308600870144
:1000F000C0308B00831203130800A0016520472045
:10010000A201A301A80120178F206E219A20A01818
:10011000B420C320E52008213821B7208428A01D61
:100120009728AC0A2208AC1FFF30A3000800220861
:10013000A3000800201C08007D0821020319080004
:10014000A10AA403031D0800A5080319A928A503F3
:100150000800A0140030A5000130A4000800A01081
:10016000FC017D08A100AA28A01040210800201C45
:10017000BE28A01B08000515A0170800A01F080036
:100180000511A0130800A901A701061BC9282914FD
:10019000A70A8519CD28A914A70A861AD1282915D6
:1001A000A70A061AD528A915A70A8518D928291635
:1001B000A70A0518DD28A916A70AA9080319080027
:1001C0002708013C031DA9170800A908031DEA28F8
:1001D00020160800201EF528AA01AB012012A91B39
:1001E00008002908A800A0120800AA0A0319AB0AEF
:1001F0002A08003C031D08002B08023C031D0800D0
:100200002908A800A016C030AA000130AB000800E1
:10021000280803190800A01128191A21A8191D215E
:10022000281A2021A81A232128182621A8183221AB
:10023000A8010800201C20174F29201C2017402946
:10024000201C20176729201C20176029201808006F
:10025000A208031908002014201BAF207D08A1006C
:10026000201308002010A01E0800A201201708007B
:10027000201C0800A208031D08002017A015322921
:100280002208031908000F3903194829A20308009E
:10029000A20E22030F399038A200A20E08002208F5
:1002A000993C0319080022080F39093C03195A29FF
:1002B000A20A0800A20E220A0F39A200A20E08000C
:1002C0000A30A7004021A703031D622908000A3055
:1002D000A7004F21A703031D69290800A701A70351
:0602E000031D6F29080058
:100E0000A60007308A00260882074034793424344B
:100E10003034193412340234783400341034083445
:0A0E200003344634213406347F34D5
:02400E00D130AF
:00000001FF
